:10000000C80800201D2A000063080000C327000064
:1000100000000000000000000000000000000000E0
:10002000000000000000000000000000870E00003B
:100030000000000000000000D7160000DF290000CB
:10004000EB2900003D2A00003F2A0000412A000061
:10005000432A0000452A0000472A0000492A0000E0
:100060004B2A00004D2A00004F2A0000512A0000B0
:10007000532A0000F1030000552A0000572A00000F
:10008000592A00005B2A00005D2A00005F2A000058
:10009000612A0000632A0000652A0000672A000028
:1000A00033030000692A00006B2A00006D2A00005B
:1000B0006F2A0000712A000011270000732A000037
:1000C00000B5010049B2002905D40121C206D20EB3
:1000D0009140BC4A116000BD00B5010049B2002941
:1000E00005D40121C206D20E9140B74A116000BD6D
:1000F00000B5010049B2002905D40121C206D20E83
:100100009140B24A116000BDF0B5020052B2002A1F
:100110001CD40322AE4B040064B2A40804256C4333
:100120001C59FF251600064008277E43B540AC4306
:100130008D01EDB20240082672439540254302002E
:1001400052B29208042462439D5022E00F24A14B36
:10015000032205006DB22540083DAE0804256E431C
:1001600005006DB22C40083CA40804256C431F59BF
:10017000FF24A44615000540082465436446AC40AE
:10018000A7438C01E4B2024008256A4394403C43F3
:100190009C51F0BD016801220A4302607047C168AA
:1001A00001220A43C260704701690800C007C00FFE
:1001B000704701210161704701690800C007C00F45
:1001C000704701210161704742698BB2134343615B
:1001D0007047016802220A430260704701680122E9
:1001E0000A430260704741688022D2000A4342609D
:1001F00070474168802252000A434260704770B4E1
:100200000022110001240300DBB25B08434005001B
:10021000EDB2AD085D400300DBB21B096B4023402B
:100220000500EDB26D080600F6B2F6086E40050056
:10023000EDB22D0975400600F6B276096E40B44362
:10024000E4019B0123431843C0B270BC704730B532
:100250000200002318001C000D00E4B2EDB2AC4215
:100260000AD21C00E4B2145D00190400A4B2FF2CF1
:1002700000DDFF385B1CEEE7C443E0B2C0B230BD26
:1002800038B586B01821002422006D46280000F001
:10029000C1FA514D40212800FFF796FF4020009001
:1002A00001200190029403946946280000F022FB8B
:1002B00007B030BD1FB50020009003904749019161
:1002C0000290474C6946200000F022FC2000FFF716
:1002D00070FF1820FFF70CFF1820FFF7FDFE02212A
:1002E0001820FFF711FF1820FFF7EAFE2000FFF7A4
:1002F00056FF2000FFF74EFF1FBD80B53948002193
:10030000017241720170FA225201C2803648817630
:1003100001713648FFF75DFF01BD324800210172CF
:1003200041720170FA225201C2802F488176017118
:10033000704710B52A4C2000FFF736FF002834D054
:100340002000FFF736FF27480178002907D0891ED3
:10035000012911D9891E19D0491E0DD025E0C18867
:10036000002905D106210170FA214901C18002E06E
:10037000C188491EC18018E04188002902D1FFF7D9
:10038000BCFF02E04188491E41800EE081880029BF
:1003900008D11548817E022901DB00218176FFF713
:1003A000ACFF02E08188491E8180C84C2000FFF725
:1003B00003FF002804D02000FFF703FF00F01EFC1D
:1003C00010BD000000E100E080E100E080E200E01C
:1003D00000E400E01CED00E0400C00407F3E000027
:1003E000008C01407400002058000020007401407F
:1003F000F8B584B08024A402B548006820400028E5
:1004000012D0B44800686946087068460078002831
:1004100005D1B148022101701021418001E0FFF7B0
:100420006CFFAB4804602DE1A9480068C00500D40A
:1004300028E1A94D2878022809D000D21EE104281D
:1004400000D1A8E014D3052800D1ECE016E1A148C2
:100450000068694608700020BB49887668460078C5
:10046000552802D10320287001E0FFF746FF09E17B
:10047000984800686946087068460078B249B24AF0
:10048000927E89188871B048807E401CAE4988767B
:10049000B54C002020702078052812D2BB48217866
:1004A0000C2251434018007A69460978884204D1E9
:1004B00068460078B649087003E02078401C207038
:1004C000E9E72078052802D1FFF717FFE9E0AF4EF2
:1004D00020780C21484330184078012818D1207822
:1004E0000C21484330188078401C68720420287022
:1004F00020780C21484330188078401CB6218900B0
:100500004843FA21490000F03DFCC01CA88041E0AE
:1005100020780C214843301840680078B2490860C0
:100520009B480078A87220780C21484330188078C6
:10053000039020780C214843301840680290AB4F5C
:100540000197039A0299019800F090FC0198207895
:100550000C21484330188178491CC9B228000A3060
:10056000FFF775FE21780C225143711889786918BC
:10057000C87220780C21484330188078401C2872BB
:100580007148297A01710121417107600020687268
:100590000520287076E06C4CA07E697A884204D3EE
:1005A0009348016802220A4302604A48006869468B
:1005B000087068460078A17E61188871A07E401C92
:1005C000A076A07E697A491C88422BDBA17E491E59
:1005D000C9B2A01DFFF73BFEA17E61184979C0B2E8
:1005E00088421DD16048694902780C235A438A1811
:1005F0009278A37E9B1E9A4202D0FFF78EFE50E0B7
:1006000002780C235A438A189578E41D00780C224E
:100610005043081846682A002100300000F026FCEC
:10062000FFF77BFE2EE02B480068694608704648BD
:1006300041790279914219D2694609780268437971
:10064000D218521E1278914207D0694801680222DE
:100650000A430260FFF761FE0FE001684279895C9E
:10066000614A11604179491C417106E060480168A6
:1006700002220A430260FFF750FE03E015480068BB
:10068000694608708020C00211490A680240002AA9
:1006900000D00860802040020A680240002A00D092
:1006A000086005B0F0BD10B5514C200000F04AFCC8
:1006B0002000FFF798FD2000FFF79BFD2000FFF7CB
:1006C0008DFD2000FFF785FD10BD0000006001409A
:1006D00008740140107401407400002070B5454852
:1006E00000240470FA214901C1804472047225007B
:1006F0002800C0B205280FD2244E2800C0B20C2119
:100700004843305CFFF77BFD2900C9B20C225143FE
:10071000711808726D1CEBE72000C0B2082811DACE
:1007200035482100C9B2405C34492200D2B2885415
:1007300033482100C9B2405C32492200D2B2885409
:10074000641CE9E770BD00005800002080B5FFF789
:10075000C5FFFFF795FDFFF7A6FF012000F0F1FCB4
:10076000FFF7A8FD01BD0000C100002080B52148B1
:100770000021017241720170FA225201C2802248A6
:10078000817601711820FFF79BFC01BD100000204D
:10079000C000002000B517480078062801D10120CC
:1007A00000E0002000BD00B500210A00D2B2082AF6
:1007B00008DA164A0B00DBB2D25C0B00DBB2C25483
:1007C000491CF2E700BD10B500210A00D2B2082A88
:1007D00008DA0A00D2B2825C0D4B0C00E4B21A5562
:1007E000491CF2E710BD0000147401407F00002096
:1007F00000740140740000202C2A0000A400002096
:10080000342A0000AC000020580000209C0000208A
:10081000000000201206130A1A43130C1A4300BFEB
:10082000094205D0830705D00270401C491EF9D14A
:10083000704700001300103906D330B414001500BF
:1008400010393CC0FCD230BC490700D30CC000D5E5
:1008500004C0890002D30280801C002900D50270E8
:100860007047FEE722490A6802430A60704702683F
:100870008BB213430360704702688BB29A430260E5
:10088000704742688BB213434360704742688BB233
:100890009A434260704782688BB21343836070470B
:1008A00082688BB29A4382607047026A8BB21343AC
:1008B00003627047026A8BB29A4302627047826A8F
:1008C0008BB2134383627047826A8BB29A4382620F
:1008D000704730B4C3680C004C4303256C43A343FA
:1008E0000C004C4354431C43C46030BC70470000B0
:1008F00034240040F8B504000D0000200700060075
:1009000063498C420BD063498C4208D062498C42C7
:1009100005D062498C4202D061498C4201D101214B
:1009200000E00100C9B2002900D1FEE729680029D2
:1009300006D0296880225202914201D2012100E0B2
:100940000100C9B2002900D1FEE76968032908D077
:100950006968002905D06968012902D069680229FF
:1009600001D1012100E00100C9B2002900D1FEE758
:10097000A968012902D0A968002901D1012100E05C
:100980000100C9B2002900D1FEE7E968002902D0C0
:10099000E968012901D1012100E00100C9B2002963
:1009A00000D1FEE76969002902D06969012901D1F6
:1009B0000120FFE7C0B2002800D1FEE78020FFF74A
:1009C00051FF2868F840002860D028680121B9400C
:1009D00001400E00002E57D06868032818D131005E
:1009E0002000FFF749FF31002000FFF74FFF3100E3
:1009F0002000FFF755FF6869012804D1310020006D
:100A0000FFF75DFF2CE031002000FFF75DFF27E0DE
:100A100031002000FFF758FF6868002804D131003A
:100A20002000FFF724FF03E031002000FFF724FF40
:100A3000A868002804D131002000FFF731FF03E04F
:100A400031002000FFF727FFE868002804D03100BC
:100A50002000FFF716FF03E031002000FFF716FF2C
:100A6000686802280BD12869012804D131002000D0
:100A7000FFF71BFF03E031002000FFF71BFF6A6850
:100A800031002000FFF725FF7F1C9AE70120F2BD0F
:100A9000000C0040400C0040800C0040C00C0040A6
:100AA000000D0040016880220A430260704701681F
:100AB00080229143016070470168022291430160E6
:100AC000704701690800C007C00F704741690122E3
:100AD0000A4342617047826A120C12040A4382621E
:100AE0007047C26A120C12040A43C26270473B4943
:100AF0000A6802430A60704739490A6802430A607B
:100B0000704738490A68384B134003430B607047FD
:100B100070B506000C0005253448864200D0FEE77B
:100B2000E06800280ED0E06880210902884209D0E0
:100B3000E068C0210902884204D0E0688021C90130
:100B4000884201D1012000E00020C0B2002800D17D
:100B5000FEE7802040022168814200D3FEE7616801
:100B6000814200D3FEE7A068012802D0A0680028D7
:100B700001D1012000E00020C0B2002800D1FEE732
:100B800080204000FFF7B3FFE068FFF7BAFF0820BE
:100B9000FFF7B2FF21683000FFF79DFF3000FFF73D
:100BA0008BFF61683000FFF79CFFA068012803D12C
:100BB0003000FFF777FF02E03000FFF778FF3000EA
:100BC000FFF784FF3000FFF77CFF002803D1002DE2
:100BD00001D06D1EF6E7012070BD000040240040EA
:100BE0004C24004044240040FF3FFFFF008C0140A4
:100BF00080B50121002000F015FB01BD50480168BF
:100C0000491C0160704738B500F032FB00F033FD3D
:100C1000002000F088FC002000F09FFC00252C0044
:100C20002000C0B20A2806DA00212000C0B200F07D
:100C3000CCFB641CF4E74348056031BD10B5404867
:100C40000168002930D00168491E01603E4C2068CF
:100C5000401C20602068052100F097F8002901D190
:100C600000F023F82068FA21890000F08EF80029AE
:100C70000AD1FFF7BDFF33490868401C08603348BC
:100C800009680170FFF79FFD2068642100F07DF87E
:100C9000002903D100F050FAFFF77CFD20682C49B1
:100CA000884201D30020206010BD70B5294C20007F
:100CB000FFF779FD002635002800C0B2082811DAB8
:100CC00020780121A940084205D001212800C0B2A6
:100CD00000F07BFB04E000212800C0B200F075FBAF
:100CE0006D1CE9E73000C0B2022813DA60780121F8
:100CF000B140084206D0012130000830C0B200F0F7
:100D000064FB05E0002130000830C0B200F05DFB5C
:100D1000761CE7E76078000603D5012000F003FCAD
:100D200002E0002000F0FFFB6078400603D50120C0
:100D300000F013FC02E0002000F00FFC70BD00008A
:100D4000B4000020BC000020B80000208C0000206F
:100D500040420F0094000020F446002804D4494289
:100D600000F013F8404260474042002905D45FD0AC
:100D700000F00BF8404249426047494200F005F854
:100D80004942604703460B43E6D40022030A8B42E4
:100D90000BD203098B4219D243088B422ED2411A3F
:100DA00000D20146524110467047FF2209023FD04F
:100DB00012068B4205D3121209028B4201D3121282
:100DC000090203098B4219D300E0090AC3098B42C7
:100DD00001D3CB01C01A524183098B4201D38B014D
:100DE000C01A524143098B4201D34B01C01A5241F0
:100DF00003098B4201D30B01C01A5241C3088B4235
:100E000001D3CB00C01A524183088B4201D38B001F
:100E1000C01A524143088B4201D34B00C01A5241C1
:100E2000884200D3401A5241CFD201461046704743
:100E300008B500F04FFC08BD70B4103A03D378C970
:100E4000103A78C0FBD2530701D318C918C001D596
:100E500008C908C0D20704D30B880380891C801CF2
:100E6000002A01D50B78037070BC70478B0701D145
:100E70008307E1D0124205D00B78491C0370401C57
:100E8000521EF9D17047FEE700B5010049B20029B2
:100E900005D40121C206D20E9140854A116000BDE1
:100EA00000B5010049B2002905D40121C206D20EC5
:100EB0009140804A116000BDF0B5020052B2002A94
:100EC0001CD403227C4B040064B2A40804256C43A8
:100ED0001C59FF251600064008277E43B540AC4349
:100EE0008D01EDB202400826724395402543020071
:100EF00052B29208042462439D5022E00F246F4BAB
:100F0000032205006DB22540083DAE0804256E435E
:100F100005006DB22C40083CA40804256C431F5901
:100F2000FF24A44615000540082465436446AC40F0
:100F3000A7438C01E4B2024008256A4394403C4335
:100F40009C51F0BDF8B58CB007001825290000248D
:100F500022006E463000FFF75DFC2900220006AD3E
:100F60002800FFF757FC3800554988420CD05549F6
:100F7000884223D05449884239D0544988424ED0BF
:100F80005349884263D084E0C020C0010090022011
:100F900001900120029003900494059469464D4805
:100FA000FFF7A8FC06940A20FFF77AFF02210A2027
:100FB000FFF782FF0A20FFF767FF6AE00C2000902E
:100FC0000220019001200290039004940594694648
:100FD0004148FFF78FFC06940B20FFF761FF0221C9
:100FE0000B20FFF769FF0B20FFF74EFF51E00320B6
:100FF000009002200190012002900390049005943B
:1010000069463648FFF776FC0C20FFF749FF0221BE
:101010000C20FFF751FF0C20FFF736FF39E00C20C2
:101020000090022001900120029003900494059406
:1010300069462A48FFF75EFC0D20FFF731FF0221C9
:101040000D20FFF739FF0D20FFF71EFF21E00120E3
:101050000090022501950294039004940594204E7B
:1010600069463000FFF746FC009501950294039411
:101070000494059469463000FFF73CFC0E20FFF70E
:101080000FFF01210E20FFF717FF0E20FFF7FCFED8
:10109000FFE79620C00107904020089009940A9429
:1010A00001200B9006A9380000F058FB0DB0F0BDF0
:1010B00000E100E080E100E000E400E01CED00E081
:1010C00000200140006801400070014000740140B0
:1010D00000780140000C0040800C0040400C0040B3
:1010E000C00C004081B0002100911F4901600168DF
:1010F000009101B0704781B00021009141688022C9
:1011000012010A4342600168009101B0704781B04A
:10111000002100914168154A0A404260016800912F
:1011200001B070471CB5040000200190009469468E
:101130000F4800F08AFC16BD80B50D48FFF7D2FFBE
:1011400001BD10B504002000C0B2002803D108483A
:10115000FFF7DDFF06E02000C0B2012802D10448FD
:10116000FFF7C9FF10BD00005A5A3412FFF7FFFF06
:1011700000140140416801220A4342607047C06880
:1011800080210840704780B586B01821002268464B
:10119000FFF740FB80200002009003200190002018
:1011A00002900390049069461C48FFF7A3FB07B028
:1011B00000BDF8B586B004000E0017002000C0B2D4
:1011C000012801D1FFF7DFFF2000C0B2012801D1C3
:1011D000012000E00020C0B205900120029000979D
:1011E00000200390049001960D4D6946280000F000
:1011F000C4FC2800FFF7BEFFFA20400000F062FDAB
:1012000007B0F0BD80B50648FFF7B9FF802801D1CF
:10121000012000E00020C0B202BD0000000C004030
:101220000028014038B505000C00002C00D1641CDA
:10123000FFF7E8FF2900C9B2884208D1002C06D088
:10124000641E002CF4D0012000F03CFDF0E7002CDF
:1012500001D1012000E00020C0B232BD42698BB252
:1012600013434361704782698BB2134383617047B4
:10127000F0B587B01821002006906C46069A200031
:10128000FFF7C8FA80273F013900C248FFF7EBFF9C
:10129000C14C20212000FFF7E6FF8021C90020007B
:1012A000FFF7E1FF8026760031002000FFF7DBFF2B
:1012B000BA4D08212800FFF7D6FF10212800FFF7BC
:1012C000D2FF40212800FFF7CEFF80218900B148DE
:1012D000FFF7C9FF802109022800FFF7C4FF04219E
:1012E0002800FFF7C0FF80214901AA48FFF7BBFF94
:1012F00001212000FFF7B7FF20212800FFF7B3FFEF
:1013000031002800FFF7AFFF009701200190002077
:1013100002900020039069469E48FFF7EBFA009781
:1013200069469C48FFF7E6FA2027009769462000A7
:10133000FFF7E0FA8020C000009069462000FFF728
:10134000D9FA009669462000FFF7D4FA08200090E9
:1013500069462800FFF7CEFA102000906946280061
:10136000FFF7C8FA4020009069462800FFF7C2FA4C
:1013700080208000009069468648FFF7BBFA8020F5
:101380000002009069462800FFF7B4FA042000909C
:1013900069462800FFF7AEFA8020400100906946B8
:1013A0007C48FFF7A7FA0120009069462000FFF76C
:1013B000A1FA009769462800FFF79CFA0096694653
:1013C0002800FFF797FA07B0F0BD38B504000D000C
:1013D0002000C0B200280FD002282BD01CD3042834
:1013E00048D037D3062861D052D308287CD06BD39D
:1013F000092800D188E095E02800C0B2002805D176
:10140000802109016348FFF72EFF04E080210901D4
:101410006048FFF723FF85E02800C0B2002804D110
:1014200020215D48FFF71FFF03E020215A48FFF706
:1014300015FF77E02800C0B2002805D18021C9003F
:101440005548FFF710FF04E08021C9005248FFF71C
:1014500005FF67E02800C0B2002805D180214900BF
:101460004D48FFF700FF04E0802149004A48FFF79C
:10147000F5FE57E02800C0B2002804D108214748F3
:10148000FFF7F1FE03E008214448FFF7E7FE49E0DB
:101490002800C0B2002804D110214048FFF7E3FE25
:1014A00003E010213D48FFF7D9FE3BE02800C0B221
:1014B000002804D140213948FFF7D5FE03E0402140
:1014C0003648FFF7CBFE2DE02800C0B2002805D13A
:1014D000802189002F48FFF7C6FE04E080218900A3
:1014E0002C48FFF7BBFE1DE02800C0B2002805D144
:1014F000802109022948FFF7B6FE04E08021090295
:101500002648FFF7ABFE0DE02800C0B2002804D14A
:1015100004212248FFF7A7FE03E004211F48FFF73C
:101520009DFEFFE731BD10B504002000C0B20028C9
:1015300009D1802149011748FFF795FE012116487E
:10154000FFF791FE08E0802149011248FFF786FE6F
:1015500001211148FFF782FE10BD38B504002000BC
:10156000C0B200280AD10D4D20212800FFF77BFED4
:10157000802149002800FFF776FE09E0074D202171
:101580002800FFF76BFE802149002800FFF766FE68
:1015900031BD0000400C0040800C0040000C0040B9
:1015A00000B5010049B2002905D40121C206D20EBE
:1015B0009140424A116000BD00B5010049B20029C6
:1015C00005D40121C206D20E91403D4A116000BDF2
:1015D000F0B5020052B2002A1CD40322394B040099
:1015E00064B2A40804256C431C59FF25160006406C
:1015F00008277E43B540AC438D01EDB2024008267A
:10160000724395402543020052B29208042462437B
:101610009D5022E00F242C4B032205006DB2254083
:10162000083DAE0804256E4305006DB22C40083C11
:10163000A40804256C431F59FF24A4461500054047
:10164000082465436446AC40A7438C01E4B20240E1
:1016500008256A4394403C439C51F0BD0168012237
:101660000A4302607047C16801220A43C2607047A2
:101670000121016170471FB50720019013480290B6
:101680000120039000200090114C6946200000F0DA
:1016900071FB2000FFF7ECFF2000FFF7E4FF1820AC
:1016A000FFF78AFF02211820FFF792FF1820FFF7AB
:1016B00077FF2000FFF7D2FF1FBD000000E100E030
:1016C00080E100E000E400E01CED00E09F0F00007E
:1016D000006001407047FEE71C490A6802430A6047
:1016E00070471B490A6802430A60704719490A6833
:1016F0000C239A4302430A60704716490A68032381
:101700009A4302430A6070470268134B13400B432D
:10171000036070470268C0239A430A43026070471F
:10172000026830239A430A4302607047016802222C
:101730000A4302607047016801220A430260704751
:101740008269120C12040A43826170473C240040F3
:101750004C24004044240040FFFEFFFFFEB505007E
:101760000C00002001006A46117107000090994E9C
:10177000B5420BD098498D4208D098498D4205D08A
:1017800097498D4202D097498D4201D1012100E055
:101790000100C9B2002900D1FEE72168002914D058
:1017A0002168012911D0216802290ED0216803295E
:1017B0000BD02168002908D02168042905D02168B0
:1017C000082902D021680C2901D1012100E0010083
:1017D000C9B2002900D1FEE7A168C02908D0A168DC
:1017E000002905D0A168402902D0A168802901D133
:1017F000012100E00100C9B2002900D1FEE7216902
:10180000002905D02169102902D02169202901D1A0
:10181000012100E00100C9B2002900D1FEE7E16822
:10182000002904D0E16880225200914201D10121B7
:1018300000E00100C9B2002900D1FEE7616900297A
:1018400008D06169022905D06169012902D0616966
:10185000032901D10120FFE7C0B2002800D1FEE733
:10186000B54224D12068FFF748FF2068002805D042
:1018700002280BD006D303280CD00FE000F060FB49
:1018800007000EE000F0ABFB07000AE000F005FBEC
:10189000070006E054480068070002E000F050FB33
:1018A000070038006168FFF770FA401E00904A4850
:1018B000854225D12068FFF719FF2068002806D04F
:1018C000042808D008280AD00C280CD00FE000F01B
:1018D00037FB07000EE000F082FB07000AE000F093
:1018E000DCFA070006E040480068070002E000F06C
:1018F00027FB070038006168FFF747FA401E009099
:10190000B54208D1802676003000FFF7E5FE3000B2
:10191000FFF7E7FE3DE03048854208D18026B6005B
:101920003000FFF7D9FE3000FFF7DBFE31E02B4837
:1019300085420DD180200001FFF7CEFE00F000FBB4
:10194000070038006168FFF720FA401E009020E091
:10195000234885420DD180204001FFF7BDFE00F0F5
:10196000EFFA070038006168FFF70FFA401E009099
:101970000FE01C4885420CD180208001FFF7ACFEAF
:1019800000F0DEFA070038006168FFF7FEF9401E3C
:101990000090012660693040002802D02800FFF73F
:1019A000CAFE207D800702D52800FFF7BFFE009900
:1019B0002800FFF7C5FEE1682800FFF7A5FEA16833
:1019C0002800FFF7A7FE21692800FFF7A9FE3000D5
:1019D000C0B2FEBD0020014000680140007001401F
:1019E00000740140007801405000002047490A6817
:1019F00002430A60704781B00021009144490160B0
:101A00000168009101B0704781B0002200924268E5
:101A100007239A430A4342600268009201B070476C
:101A200081B001000020009088680005000D0A6860
:101A3000009201B0704781B0002200920A05120D99
:101A4000C2600268009201B07047F8B506000C0051
:101A50000020050001210F0000902E4A964200D080
:101A6000FEE762682C4B9A4200D3FEE72268002A08
:101A700014D02268012A11D02268022A0ED02268CE
:101A8000032A0BD02268042A08D02268052A05D030
:101A90002268062A02D02268072A01D10800FFE73F
:101AA000C0B2002800D1FEE72020FFF79FFF3000E2
:101AB000FFF7A1FF21683000FFF7A6FF3000FFF716
:101AC000AFFF00906068002819D0009800280BD163
:101AD0003000FFF7A5FF012811D02800451CFA218E
:101AE000490088420BD2F3E73000FFF799FF002846
:101AF00005D02800451CFA2149008842F4D36168CA
:101B00003000FFF798FF3800C0B2F2BD3424004027
:101B10005A5A341200140140FF0F000067490A6846
:101B200002430A6070470268F0239A430A43026046
:101B30007047016808220A43026070470168082262
:101B4000914301607047026804239A430A4302608C
:101B50007047026803239A430A4302607047416852
:101B600002220A4342607047416802229143416069
:101B700070474A07520F0261704738B504000D00E4
:101B80004F48844200D0FEE72968042905D029681F
:101B9000022902D02968012901D1012100E0002198
:101BA000C9B2002900D1FEE7696800292CD0696814
:101BB000102929D06968202926D06968302923D0C6
:101BC0006968402920D0696850291DD0696860295A
:101BD0001AD06968702917D06968802914D069689B
:101BE000902911D06968A0290ED06968B0290BD05E
:101BF0006968C02908D06968D02905D06968E029DA
:101C000002D06968F02901D1012100E00021C9B2A8
:101C1000002900D1FEE7E968002902D0E96804291B
:101C200001D1012100E00021C9B2002900D1FEE765
:101C30002969002908D02969012905D029690229C3
:101C400002D02969032901D1012100E00021C9B294
:101C5000002900D1FEE784420FD180204000FFF729
:101C60005DFF29682000FFF784FF69682000FFF707
:101C70005AFFA868012806D101E000201CE02000DE
:101C8000FFF757FF02E02000FFF758FFE968200048
:101C9000FFF759FFE868042803D129692000FFF7FE
:101CA00058FF6869012803D12000FFF758FF02E0C0
:101CB0002000FFF759FF012032BD0000342400400E
:101CC0000028014010B504000C4800680C49FFF7DB
:101CD0005CF860430B49884202D380204004FFE750
:101CE000411E094A11600021084A1160084909682B
:101CF0000A00D203D20F002AF8D010BD54000020F1
:101D000040420F000100000114E000E018E000E094
:101D100010E000E0016880220A4302607047016819
:101D20008022914301607047016802229143016063
:101D3000704701690800C007C00F70474169012260
:101D40000A4342617047826A81627047C26AC16217
:101D5000704736490A6802430A60704734490A6886
:101D600002430A60704733490A68334B1340034308
:101D70000B60704770B506000C0005252F488642A1
:101D800000D0FEE7206800280ED02068802189015D
:101D9000884209D02068C0218901884204D0206887
:101DA00080214901884201D1012000E00020C0B219
:101DB000002800D1FEE7E068012802D0E068002892
:101DC00001D1012000E00020C0B2002800D1FEE7D0
:101DD0000120FFF7BEFF2068FFF7C5FF0420FFF7D3
:101DE000BDFF61683000FFF7AEFF3000FFF79CFFDA
:101DF000A1683000FFF7AAFFE068012803D1300096
:101E0000FFF788FF02E03000FFF789FF3000FFF79F
:101E100095FF3000FFF78DFF002803D1002D01D082
:101E20006D1EF6E7012070BD000000004024004058
:101E30004C24004044240040FFCFFFFF00600140DD
:101E400098480168E020C002084070479548016842
:101E5000E020C00008407047924800684007400FEB
:101E6000704791480168F0200003084070478F4890
:101E700000680221084070478C480068000C40064A
:101E8000400E7047894801687020084070478848B4
:101E90000168C02080020840704710B50024FFF799
:101EA000DBFF00280AD001280BD002280CD0042820
:101EB0000DD005280ED006280FD011E000F08FF8C5
:101EC00010E07C4800680DE000F0A6F80AE000F0A1
:101ED00064F807E07848006804E08020000201E030
:101EE00000F07DF810BD10B50024FFF7AFFF00280B
:101EF00010D08021C90088420FD0A021C90088429B
:101F00000FD0C021C90088420FD0E021C90088420B
:101F10000FD012E0FFF7C1FF11E0FFF7BEFF40084E
:101F20000DE0FFF7BAFF800809E0FFF7B6FFC00831
:101F300005E0FFF7B2FF000901E0FFF7AEFF10BDBB
:101F400010B50024FFF77CFF002810D08021C902C3
:101F500088420FD0A021C90288420FD0C021C902F7
:101F600088420FD0E021C90288420FD012E0FFF76B
:101F7000BAFF11E0FFF7B7FF40080DE0FFF7B3FF2E
:101F8000800809E0FFF7AFFFC00805E0FFF7ABFFEF
:101F9000000901E0FFF7A7FF10BD10B50024FFF70F
:101FA00076FF00280CD08021490288420BD0802186
:101FB000890288420AD0C0218902884209D00BE0F8
:101FC000962000030AE09620800207E09620400257
:101FD00004E09620000201E09620000310BD10B539
:101FE0000024FFF73EFF00280CD0802149028842E0
:101FF0000AD080218902884208D0C0218902884203
:1020000006D007E02D4806E02D4804E02D4802E008
:102010002D4800E0294810BD70B500242500FFF7C9
:1020200026FF002802D0022804D006E0FFF7D7FFE1
:10203000060005E01F48066802E0FFF7D0FF060033
:10204000FFF720FF00280ED010280DD020280DD03B
:1020500030280DD040280DD0502811D0602811D044
:10206000702815D016E015E0760813E0B60811E0E8
:10207000F6080FE030000C21FEF787FE060009E0AD
:10208000360907E030001821FEF77FFE060001E068
:102090007609FFE7FFF7F0FE0100491C4E433000D0
:1020A00070BD000000240040042400400C240040C7
:1020B00024240040500000204C00002000127A0030
:1020C0000024F40000366E010048E80130B500201D
:1020D00001246D4D296849082140002902D00129B9
:1020E00018D01AE069490968090C0907090F012984
:1020F00004D00CD3032907D003D308E064490800B7
:1021000007E06449080004E06349080001E063490E
:10211000080002E09A490968080029680909490786
:10212000490F00290BD002290FD00CD3042910D05D
:102130000DD3062913D010D3072914D014E02100A1
:10214000FEF723FE10E040080EE080080CE0C00817
:102150000AE00C21FEF719FE06E0000904E0182150
:10216000FEF713FE00E040092968090C4906490EF4
:10217000491C48432968C9080C40002C01D00221A1
:10218000484330BD38B507247E4D286820400128DB
:1021900008D002280BD004280ED005282DD0062800
:1021A00030D034E076480068774908604AE0FFF7AD
:1021B0008DFF7549086045E074480068000C800791
:1021C000800F002805D002280DD007D303280FD098
:1021D00012E0962000036C4908600DE09620800212
:1021E0006949086008E0962040026749086003E0FA
:1021F000962000026449086024E06548006862494E
:1022000008601FE0FA20C0015F4908601AE01F481B
:102210000068000C0007000F012804D00FD303282A
:1022200009D004D30BE01A48574908600AE019485E
:102230005549086006E018485349086002E017480D
:10224000514908602868000A0440042C06D019D3BC
:10225000062C0DD007D3072C0FD013E04A48016895
:10226000490801600EE0484801688908016009E0FA
:1022700045480168C908016004E04348016809094C
:102280000160FFE731BD00000C2400400424004041
:102290000024F40000366E010048E80100127A00C4
:1022A00080B53C480168802252010A4302600168FF
:1022B00080220A430260032037490A6802430A6009
:1022C0000A22364B1A6000220A602E490A6852011F
:1022D00052090A605521324A116032490860324879
:1022E0000168090C0268D3439AB2914201D1006897
:1022F00002E02E48008880B2C006C00E2C4908605B
:102300002C480168090C0268D3439AB2914201D16A
:10231000006802E02848008880B2C0B227490860FF
:1023200027480168090C0268D3439AB2914201D14F
:10233000006802E02348008880B2C0B222490860E9
:1023400022480168090C0268D3439AB2914201D134
:10235000006802E01E48008880B2C0B21D490860D3
:102360001D480168C02252000A43026005201B4933
:10237000086001201A490860FFF704FF01BD000052
:10238000500000200024004054000020242400407D
:102390004C0000203424004000E0014004F80140DB
:1023A0001C2400400400004098FAFF1FAAFBFF1FF6
:1023B0003820004040FBFF1FC2FBFF1F08240040E5
:1023C00044FBFF1FC0FBFF1F2824004020FBFF1F12
:1023D000CEFBFF1F14240040C40C00400028004026
:1023E00004280040426807239A430A43426070472A
:1023F00096490A6807239A4302430A607047944942
:102400000A68944B134003430B60704799490A686C
:10241000FF239A4302430A607047026803239A43EA
:102420000A430260704742698BB2134343617047AD
:1024300082698BB213438361704738B504008E4DB7
:1024400002212800FFF7E9FF200000280CD080219E
:102450004902884221D080218902884236D0C02199
:10246000890288424BD063E084480168090C026805
:10247000D3439AB2914201D1006802E080480088BB
:1024800080B2C0B2FFF7C2FF00212800FFF7C5FFEE
:1024900000217C48FFF7A6FF62E07B480168090C39
:1024A0000268D3439AB2914201D1006802E07748B2
:1024B000008880B2C0B2FFF7A9FF00212800FFF713
:1024C000ACFF01216F48FFF78DFF49E070480168BC
:1024D000090C0268D3439AB2914201D1006802E02C
:1024E0006C48008880B2C0B2FFF790FF002128003E
:1024F000FFF793FF02216348FFF774FF30E066485F
:102500000168090C0268D3439AB2914201D1006874
:1025100002E06248008880B2C0B2FFF777FF012175
:102520002800FFF77AFF02215648FFF75BFF17E00C
:1025300052480168090C0268D3439AB2914201D112
:10254000006802E04E48008880B2C0B2FFF75EFF2C
:1025500000212800FFF761FF00214A48FFF742FFF2
:102560002000FFF74CFF0020FFF742FF31BDF0B520
:1025700087B00520694608761821002422006D46A0
:102580002800FEF747F9464D80273F013900280013
:10259000FFF74EFF802189002800FFF749FF8026C2
:1025A000F60031002800FFF743FF802149003D4835
:1025B000FFF73EFF009701270197029403946946B5
:1025C0002800FEF797F98020800000900197029480
:1025D000039469462800FEF78DF90096019702944E
:1025E000039469462800FEF785F98020400000909A
:1025F00001970294039469462A48FEF77BF931005B
:102600002800FFF710FF31002800FFF70CFF310012
:102610002800FFF708FF009601970294039469468B
:102620002800FEF767F90096019702940394694623
:102630002800FEF75FF9009601970294039469461B
:102640002800FEF757F907B0F0BD00000024004055
:1026500004240040FFFFF0FF80B5C0208002FFF798
:10266000ECFEFFF784FF802149000E48FFF7DBFEF8
:1026700001BD0000082400400010004040FBFF1F87
:10268000C2FBFF1F00E001403CFBFF1FC4FBFF1F1C
:1026900038FBFF1FC6FBFF1F34FBFF1FC8FBFF1FDC
:1026A000400C0040800C004000B5010049B20029F8
:1026B00005D40121C206D20E9140374A116000BDF7
:1026C00000B5010049B2002905D40121C206D20E8D
:1026D0009140324A116000BD00B502690A40002AEB
:1026E00001D0816100E0416100BD42698BB21343BA
:1026F0004361704730B483680C004C4303256C433E
:10270000A3430C004C4354431C43846030BC7047CB
:10271000F8B51024244F3868204000283AD0204DC6
:102720008026360131002800FFF7D6FF1F480168D8
:10273000302291430160016820220A4302601C4854
:1027400001680422914301601A48016801600D206C
:10275000FFF7B6FF0D20FFF7A7FF17480168022219
:102760000A43026031002800FFF7B6FFFDF7FEFFC5
:102770008021C9002800FFF7B8FF31002800FFF7CB
:10278000ABFF3C60032210210648FFF7B3FF1E2079
:10279000FFF796FFF1BD000000E100E080E200E0FD
:1027A000400C0040C00D0040D40D00404C0C0040D7
:1027B000600C004008740140007401400349C1608E
:1027C000704780B50248FFF7F9FF01BDBBAA5C5C0A
:1027D0000028004080B50320FEF7A4FC00F01AF8A2
:1027E000042250210020FEF7E4FCFA21C900012058
:1027F000FEF718FD0028F8D0042000F01AF800F0C9
:1028000035F8FFF729FFFDF7A1FFFEF7FCF9FEF70A
:1028100015FAFCE780B500F039F801BD42680C23D9
:102820009A430A43426070474168012291434160E4
:10283000704738B50400044D21002800FFF7EEFF73
:102840002800FFF7F1FF31BD002800400D490A685C
:1028500002430A6070470B490A6882430A60704766
:10286000026B520A52020A430263704780B5042089
:10287000FFF7ECFF00210448FFF7F2FF0420FFF709
:10288000EAFF01BD34240040001001400448016803
:1028900004220A430260016801220A430260704771
:1028A00010E000E01234567800000000112233449A
:1028B00055667788100102009C000020000000008F
:1028C0002000080000000020000000002100080097
:1028D000080000200000000030000800A4000020D4
:1028E0000000000031000800AC00002000000000E3
:1028F0000080000000127A0000127A0070B40121FA
:10290000002213E00368001D0B4202D04D46EB1875
:102910005B1E1A601B1D241F042CFAD21D00A60783
:1029200001D51A80AD1C0C4000D02A700468001D2F
:10293000002CE7D170BC704730B401210EE0036871
:10294000C318446808300C4202D04D462C19641E4E
:102950001D6825601B1D241D121FF9D10268001D72
:10296000002AECD130BC704710B5074979441831C2
:10297000064C7C44163404E0081D0A688918884710
:102980000100A142F8D110BD08000000280000009D
:102990006DFFFFFF6C0000005800002000000000E9
:1029A00099FFFFFF58000000FCFEFFFF0000002021
:1029B0000000000000F00DF8002801D0FFF7D4FF60
:1029C00000BF00BF002000BF00BFFFF703FF00F003
:1029D00002F80120704780B500F002F801BDFEE763
:1029E0000746384600F002F8FBE7FEE780B500BF77
:1029F00000BF024A11001820ABBEFBE72600020010
:102A00000548014603B4684680F3098800BF00BF4B
:102A100000BF00BFFFF7CEFFA5EDF5FE01488047E0
:102A200001480047A1220000012A0000535730311D
:102A3000303120203230323530323138FEE7FEE797
:102A4000FEE7FEE7FEE7FEE7FEE7FEE7FEE7FEE75E
:102A5000FEE7FEE7FEE7FEE7FEE7FEE7FEE7FEE74E
:102A6000FEE7FEE7FEE7FEE7FEE7FEE7FEE7FEE73E
:042A7000FEE7FEE798
:0400000500002A01CC
:00000001FF
